:1000000010C42AC429C428C425C726C425C424C4AE
:1000100023C4D4C621C420C41FC41EC41DC41CC410
:100020001BC43F3F3F3F3F3F3F3F3F3F3F3F3F3F7F
:100030003F3F3F3F3F3F3F3F3F3F3F3F3F3F3F3FD0
:100040003F3F3F3F3F3F3F3F3F3F3F3F3F3F3F3FC0
:100050003F3F3F3F3F3F3F3F3F3F3F3F3F3F3F3FB0
:100060003F3F3F3F3F3F3F3F3F3F3F3F3F3F3F3FA0
:100070003F3F3F3F3F3F3F3F3F3F3F3F3F3F3F3F90
:100080003F3F3F3F3F3F3F3F3F3F3F3F3F3F3F3F80
:100090003F3F3F3F3F3F3F3F3F3F3F3F3F3F3F3F70
:1000A0003F3F3F3F3F3F3F3F3F3F3F3F3F3F3F3F60
:1000B0003F3F3F3F3F3F3F3F3F3F3F3F3F3F3F3F50
:1000C0003F3F3F3F3F3F3F3F3F3F3F3F3F3F3F3F40
:1000D0003F3F3F3F3F3F3F3F3F3F3F3F3F3F3F3F30
:1000E0003F3F3F3F3F3F3F3F3F3F3F3F3F3F3F3F20
:1000F0003F3F3F3F3F3F3F3F3F3F3F3F3F3F3F3F10
:100100003F3F3F3F3F3F3F3F3F3F3F3F3F3F3F3FFF
:100110003F3F3F3F3F3F3F3F3F3F3F3F3F3F3F3FEF
:100120003F3F00000000000000000404040404003D
:1001300004000A0A000000000000000A1F0A1F0A4B
:100140000000040F140E05150E04181902040813FC
:1001500003000C12140815120D0004040000000026
:100160000000020408080804020008040202020455
:1001700008000004150E150400000004041F040408
:10018000000000000000000C0C100000001F000028
:10019000000000000000000C0C0001010202040439
:1001A00008080E11131519110E00040C04040404A0
:1001B0000E000E11010204081F000E1101060111AC
:1001C0000E0002060A121F0202001F101E0101117A
:1001D0000E000E11101E11110E001F010102040469
:1001E00004000E11110E11110E000E11110F01114C
:1001F0000E0000000C0C000C0C0000000C0C000C9D
:100200000C10020408100804020000001F001F0068
:10021000000008040201020408000E11010204009B
:1002200004000E11131517100F000E11111F1111DC
:1002300011001E11111E11111E000E1110101011AF
:100240000E001E11111111111E001F10101E101092
:100250001F001F10101E101010000E11101311118E
:100260000E001111111F111111000E0404040404D9
:100270000E000101010111110E00111214181412C7
:1002800011001010101010101F00111B1515111166
:10029000110011191513111111000E111111111165
:1002A0000E001E11111E101010000E11111111114F
:1002B0000E011E11111E111111000E11100E01114F
:1002C0000E001F0404040404040011111111111183
:1002D0000E0011111111110A040011111111151B39
:1002E0001100110A0404040A11001111110A040476
:1002F00004001F01020408101F000C080808080869
:10030000080C10100808040402020602020202028D
:100310000600040A000000000000000000000000C9
:10032000001F080400000000000000000E1111135F
:100330000D0010101E1111111E0000000E111010E2
:100340000F0001010F1111110F0000000E111F10FD
:100350000F0003040E040404040000000F11110F29
:10036000010E10101E1111111100040004040404E8
:1003700004000400040404040418101012141C12D5
:100380001100040404040404020000001E151515E5
:100390001500000016191111110000000E111111A5
:1003A0000E0000001E111119161000000E1111137D
:1003B0000D01000016191010100000000F100E01A2
:1003C0001E0004040E0404040300000011111113A4
:1003D0000D0000001111110A04000000151515157B
:1003E0000A000000110A040A110000001111110F87
:1003F000010E00001F0204081F0002040408040488
:1004000002000404040404040404080404020404B0
:1004100008000D160000000000000A150A150A1554
:100420000A1506091E081E0906000000000000004B
:1004300000000000000000000000000000000000BC
:1004400000000000000000000000000000000000AC
:10045000000000000000000000000000000000009C
:10046000000000000000000000000000000000008C
:10047000000000000000000000000000000000007C
:10048000000000000000000000000000000000006C
:10049000000000000000000000000000000000005C
:1004A000000000000000000000000000000000004C
:1004B000000000000000000000000000000000003C
:1004C000000000000000000000000000000000002C
:1004D000000000000000000000000000000000001C
:1004E000000000000000000000000000000000000C
:1004F00000000000000000000000000000000000FC
:1005000000000000000000000000000000000000EB
:1005100000000000000000000000000000000000DB
:1005200000000000000000000000040004040404B7
:10053000040000010E1314180E100609081E080806
:100540000916110E1111110E110011110A1F041FAD
:10055000040E040404000004040407080E11110E24
:10056000021C000A0000000000000E1117191711EC
:100570000E000E020A0E000E000000000912120901
:1005800000000000001F010000000000000E00003D
:1005900000000E111D1B1D1B0E00000E00000000B0
:1005A00000000C120C000000000000041F04001FDB
:1005B0000000180408101C000000180408041800AB
:1005C00000000E0C100000000000000011111119B5
:1005D00016100F1D1D1D0D0505050000000400006F
:1005E0000000000000000004020C081808081C00AD
:1005F00000000C120C001E0000000000120909127D
:10060000000011111204090B1711111112040E0927
:100610001217190D0E1C090B171104000402011109
:100620000E000C020E111F11110006080E111F11F1
:100630001100040A0E111F1111000D160E111F11C9
:1006400011000A000E111F1111000E110E111F11C1
:1006500011000B1414171C1417000E111010101198
:100660000E180C021F101E101F0006081F101E106F
:100670001F00040A1F101E101F000A001F101E106A
:100680001F000C020E0404040E0006080E040404ED
:100690000E00040A0E0404040E000A000E040404F2
:1006A0000E001E09091D09091E000D16111915134A
:1006B00011000C020E1111110E0006080E1111117D
:1006C0000E00040A0E1111110E000D160E1111115B
:1006D0000E000A000E1111110E0000110A040A1179
:1006E0000000010F131515191E100C021111111124
:1006F0000E000608111111110E00040A111111113A
:100700000E000A00111111110E00060811110A0441
:1007100004001C080E09090E081C0E111E121111EE
:1007200012000C020E1111130D0006080E11111FFC
:100730000F0F040A0E11113F3D3C0D160E1111133F
:100740000D000A000E11113F3F3F0E110E11113323
:100750003D3000000E1516170F0300000E11103F5C
:100760003F3F0C020E111F100F0006080E111F1F35
:100770000F0F040A0E111F3C3F3C0A000E111F1000
:100780000F000C020004043F3F3F0608000404343D
:100790003430040A000404070703000A0004043F7D
:1007A0003F3F1B0C120E11110E000D160016191FE3
:1007B0001F0F0C020E11113D3E3C06080E111111C7
:1007C0000E00040A0E11113F3F3F0D160E1111319C
:1007D0003E300A000E1111130F030004001F003FEA
:1007E0003F3F00010E1111110E100C021111111FCB
:1007F0000F0F06081111113F3D3C040A111111138E
:100800000D000A001111113F3F3F06081111113F61
:10081000313E10101C12121F13130A001111113F48
:100820003F3F11241FBECFE5D2E0DEBFCDBF10E0B9
:10083000A0E6B0E0EAE6F1E102C005900D92A23632
:10084000B107D9F711E0A2E6B0E001C01D92A636CB
:10085000B107E1F702D088C4D3CB2F923F925F92C9
:100860006F927F928F929F92AF92BF92CF92DF92C0
:10087000EF92FF920F931F93CF93DF93CDB7DEB725
:1008800021970FB6F894DEBF0FBECDBF8EEF82BBAF
:100890004BD183E390E0B3D28090600090906100F0
:1008A0002224332455246624EFEF7E2E7FEFC72EBB
:1008B00005C0552402C0552401C06624ADD2082FBE
:1008C000803280F09101472D662D852D47D126E09D
:1008D000520E3AEF351590F788E0680EE7EFE6150F
:1008E00040F3E9CF813029F38230B1F495D2C82E9C
:1008F00093D2082F91D2282F1127C801807E9070A3
:1009000064E070E00AD4C694C694C694C694C694B3
:10091000207CC22AC62AD2CF833019F47DD2C82EB9
:10092000CDCF8430B1F478D2782E76D2082F74D21D
:10093000282F1127C801807E907064E070E0EDD30D
:1009400076947694769476947694207C722A762A9D
:10095000B5CF853019F460D2782EB0CF8630D1F47F
:100960005BD2082F59D2E82E57D2282FFF24C70177
:10097000807E907064E070E0D0D31B0102950695F4
:10098000077011273327207C3070022B132B202A6D
:10099000312A94CF873021F43FD2282E33248ECFB2
:1009A000883091F4FAEF5F0E26EF2515D8F438EF72
:1009B000630E80EF861518F066EF562E13C056EFC3
:1009C000552E40EF642E0EC0893009F477CF8A305F
:1009D00039F4E8E06E0EFBEFF61508F46ECF6ECF3B
:1009E0008B3039F400E29101472D662D852DB6D06C
:1009F00065CF8C3051F4F401C401805094401192C1
:100A0000E817F90709F455CFFACF8D3009F453CF21
:100A10008E3069F401D2E82EFFD1F82EFDD1182FC7
:100A2000FBD10C2D282F412F6F2D8E2D65C08F30BF
:100A300069F4F2D1182FF0D1E82FFF27FE2FEE270F
:100A4000E80DF91DE10FF11DC08238CF803129F585
:100A5000E3D1A82EE1D1B82EDFD1D82EDDD1E82EFA
:100A6000FF240DC09983D8D19981F801E90FF11DB8
:100A7000EA0DF11D80839F5F9D15A1F7F394FE148D
:100A800009F41CCF2F2D2B0D312D311DC901182F2D
:100A90000027080D191D90E0EFCF813149F4BCD13A
:100AA000582EBAD1682E3BEF381708F406CF06CF80
:100AB000823121F4212C81E0382E00CF8331F1F4F2
:100AC000ABD1D82EA9D1E82EA7D1182FA5D1F82EB9
:100AD0000C2D2E2D412F6E2D8D2D4FD12F2D412FD1
:100AE0006E2D812F4AD12F2D4D2D6F2D812F45D168
:100AF0002E2D4D2D6F2D8D2D40D1E0CE843109F05E
:100B0000DDCE8AD1D82E88D1182F86D1E82E84D177
:100B1000F82E07C00C2D212F4E2D612F8D2D2DD19C
:100B20001F5FF116B8F7CACEF89480E885BF8FEF43
:100B300086B980E094E095BD84BD8BE490E099BDDA
:100B400088BD82E890E09BBD8ABD83E38FBD89E0CC
:100B50008EBD80E489BF88BF789408950F931F935A
:100B6000CF93DF93582FE9016D3F88F5E02FFF27E2
:100B700073E0EE0FFF1F7A95E1F7EE5DFF4F20E087
:100B800030E0862F9927052F1127782F6627605090
:100B90007C4F549180E090E0D801A60FB71F55FF1D
:100BA00002C04C9305C0CF3FD10509F008F4CC93A7
:100BB000019611968630910511F0550FF0CF2F5FF9
:100BC0003F4F60507F4F31962830310511F7DF914C
:100BD000CF911F910F9108956C3F48F4E62FFF27A6
:100BE000FE2FEE27E050FC4FE80FF11D40830895E3
:100BF00090E08FEF09C0E82FFF27FE2FEE27E0508F
:100C0000FC4FE90FF11D10829150A9F78150E1F7D7
:100C100008957F928F929F92AF92BF92CF92DF9270
:100C2000EF92FF920F931F93CF93DF93D82EC62E90
:100C3000902E042F1127081B1109C22FDD27C61B78
:100C4000D109101611061CF451E0752E05C010953F
:100C500001951F4F4FEF742E1C161D061CF431E03A
:100C6000832E05C0D095C195DF4F2FEF822E492DE1
:100C70006C2D8D2DB1DF0C171D0744F47801EE0C9F
:100C8000FF1CAD2CBC2CCC24DD242EC07E01EE0C30
:100C9000FF1CAD2CBC2CCC24DD2410C0EC0EFD1EA2
:100CA000E016F1061CF0E01AF10AB80CA70C492D69
:100CB0006B2D8A2D91DF0894C11CD11C8C2D992796
:100CC000801791075CF315C0E00EF11EEC16FD06CF
:100CD0001CF0EC1AFD0AA70CB80C492D6B2D8A2DBF
:100CE0007BDF0894C11CD11C8C2D99278C179D0784
:100CF0005CF3DF91CF911F910F91FF90EF90DF9008
:100D0000CF90BF90AF909F908F907F900895FF926B
:100D10000F931F93CF93DF93F62E042F122FC82F1C
:100D2000DD2705C0412F602F8C2F56DF21968F2D98
:100D300099278C179D07B0F7DF91CF911F910F91E5
:100D4000FF900895FF920F931F93CF93DF93F82E98
:100D5000042F122FC62FDD2705C0412F6C2F8F2D9A
:100D60003BDF2196802F99278C179D07B0F7DF91E5
:100D7000CF911F910F91FF9008950F93582F342F0B
:100D8000422F621759F4381718F49927532F382F28
:100D9000202F462F632F852FBADF0EC0831751F403
:100DA000261720F4862F9927622F482F202F852F72
:100DB000C9DF02C0432F2DDF0F9108951F920F92BC
:100DC0000FB60F9211248F939F93EF93FF939CB1D3
:100DD0007894E0916201EF5F80916301E81731F050
:100DE000E0936201FF27EE59FF4F9083FF91EF914F
:100DF0009F918F910F900FBE0F901F90189510929A
:100E0000620110926301292F332720BD89B980E93F
:100E10008AB986E880BD089590916201809163014E
:100E20009817D1F3E0916301EF5FE0936301FF272F
:100E3000EE59FF4F8081992708959091620180912A
:100E4000630120E0981709F421E081E02827822F30
:100E5000992708950F930FB70F93EF93FF931F9365
:100E600010916401112309F03CC1ECB5FDB506E613
:100E7000E00F07E0F01FE45BF04009940000000081
:100E80000000000000000000000000000000000062
:100E90000000000000000000000000000000000052
:100EA0000000000000000000000000000000000042
:100EB0000000000000000000000000000000000032
:100EC000000000000000000000000000F09165013B
:100ED000EE273898019101910191019101910191C1
:100EE0000191019101910191019101910191019172
:100EF0000191019101910191019101910191019162
:100F00000191019101910191019101910191019151
:100F10000191019101910191019101910191019141
:100F20000191019101910191019101910191019131
:100F30000191019101910191019101910191019121
:100F40000191019101910191019101910191019111
:100F50000191019101910191019101910191019101
:100F600001910191019101910191019101910191F1
:100F700001910191019101910191019101910191E1
:100F800001910191019101910191019101910191D1
:100F900001910191019101910191019101910191C1
:100FA00001910191019101910191019101910191B1
:100FB00001910191019101910191019101910191A1
:100FC0000191019101910191019101910191019191
:100FD0000191019101910191019101910191019181
:100FE0000191019101910191019101910191019171
:100FF0000191019101910191019101910191019161
:101000000191019101910191019101910191019150
:101010000191019101910191019101910191019140
:101020000191019101910191019101910191019130
:101030000191019101910191019101910191019120
:101040000191019101910191019101910191019110
:101050000191019101910191019101910191019100
:1010600001910191019101910191019101910191F0
:1010700001910191019101910191019101910191E0
:1010800001910191019101910191019101910191D0
:1010900001910191019101910191019101910191C0
:1010A00001910191019101910191019101910191B0
:1010B00001910191019101910191019101910191A0
:1010C0000191019101910191019101910191019190
:1010D00001910191389AF0936501FF23A9F411E081
:1010E00013C01395103129F0143131F01C3338F44A
:1010F0000BC003E20FBD08C003E30FBD05C01127FD
:10110000F4E0F093650100C0109364011F91FF911A
:10111000EF910F910FBF0F91189597FB092E07269E
:101120000AD077FD04D00CD006D000201AF47095B8
:1011300061957F4F0895F6F7909581959F4F08959B
:10114000AA1BBB1B51E107C0AA1FBB1FA617B707ED
:1011500010F0A61BB70B881F991F5A95A9F7809509
:0A1160009095BC01CD010895FFCF6A
:02116A0000047F
:00000001FF
